:020000040800F2
:10000000D80A0020D9000008DD340008D12C0008EF
:1000100000000000000000000000000000000000E0
:10002000000000000000000000000000E1340008B3
:100030000000000000000000DF340008E334000886
:10004000EB00000800000000EB000008EB000008D7
:10005000EB000008EB000008890900089F09000870
:1000600000000000C1080008D1080008EB000008EB
:10007000EB000008EB000008EB00000800000000A7
:10008000EB0000080000000000000000EB0000088A
:1000900000000000EB000008EB000008EB00000887
:1000A000EB000008EB000008EB0000088D3F0008A3
:1000B000EB0000080000000000000000000000004D
:1000C0000448854600F06AF900480047C542000828
:1000D000C046C046D80A002004488047044800476C
:1000E000FEE7FEE7FEE7FEE7FEE7FEE7D3350008A2
:1000F000C100000830B50B46014600202022012433
:1001000009E00D46D5409D4205D31D469540491B4B
:100110002546954040191546521E002DF1DC30BD94
:1001200070B500242546002801DA01244042002948
:1001300001DA01254942FFF7DDFFAC4200D0404221
:10014000002C00D0494270BD03460B439B0703D0EF
:1001500009E008C9121F08C0042AFAD203E00B788C
:100160000370401C491C521EF9D27047D2B201E004
:100170000270401C491EFBD270470022F6E710B502
:1001800013460A4604461946FFF7F0FF204610BD05
:10019000421C0178401C0029FBD1801A7047F8B539
:1001A00002464A40D40F42004B0052085B089A4274
:1001B00002D20246084611464A0023D0C30D4A0027
:1001C000DDB2120EAD1A202D35DA49020126490A98
:1001D000F6058A19002C00D0524220214F1B1146EF
:1001E000B9402A411018C20D9A4221D0002C17D0D4
:1001F000012D08DCDA05801AD20F8019D207DBB294
:1002000000F092F8F8BDDA05801A012340001B06C1
:10021000C01880185A428018CA0F1043490007E0DE
:100220004908C2071143DA05801A8019400880186E
:1002300000F072F8F8BD61000122511A001BF7E7C7
:100240000122D2075140AAE70122D2075040A6E777
:10025000024670B54A40D30FDB0740002DD04A005C
:100260002AD0010E140E000212020919400A520A85
:100270008418E50104465443000A120A2E04504330
:10028000A4194219200CC543AA18120C0125AD036C
:10029000521C521912047F39240400D0521C1043FE
:1002A00001D44000491EC2B20C06C0092018401CEF
:1002B0004008802A02D003E0002070BD40084000C2
:1002C000002900DA0020184370BD420005D042002A
:1002D000120E52428A4201DB00207047C9050818FD
:1002E000704710B500229623114600F01DF810BD8E
:1002F000410040020122400AD205090E80187F29E0
:1003000001DA00207047962903DC9622511AC84072
:100310007047963988407047002904DA401C49002C
:1003200001D140084000704770B40024050C05D18D
:100330001024000402D1002921D01124050E01D17E
:1003400000020834050F01D10001241D850F01D1E1
:100350008000A41C002801DB4000641C002908D098
:1003600020252E1B0D46F540A14000D00121294338
:10037000084301061B1B000ADB1D02D5002070BCD0
:100380007047DB05181880180029F8DA401C49006E
:10039000F5D170BC4008400070470000064C0125B4
:1003A000064E05E0E36807CC2B430C3C984710341D
:1003B000B442F7D3FFF788FE7C4700089C4700084B
:1003C00070B50446006802F0A1FD002824D0206822
:1003D00081688907C90F04D18168104A1140103122
:1003E000816001F071FA054612E001F06DFA401BE0
:1003F00002280DD920688068400709D5A06D10211A
:100400000843A065E06D01210843E065084670BD22
:10041000206880684007E8D4002070BDE8FFFF7FB7
:1004200010B5846AA16D502211420DD1A06D012139
:1004300049020843A065206802F06CFD00281AD02C
:10044000A07E002807D016E0A16DC90623D520465E
:1004500000F038FC10BD2068016809070BD502F0D8
:1004600055FD012200280AD0A06D20210843A06577
:10047000E06D1043E065204600F022FC10BD2068CE
:1004800041680C2399434160A06DFF2101318843ED
:100490001043A065EFE7216D496B884710BD10B58B
:1004A000806A816D402211438165C16D0422114330
:1004B000C16500F007FC10BD10B5806A00F001FCBA
:1004C00010BD0000F8B50446006881688907CD0FAB
:1004D00002F018FD00282AD0002D28D1206881685C
:1004E0000522114010260127012914D18168114AE3
:1004F0001140891C816021680320086001F0E4F943
:10050000054610E001F0E0F9401B02280BD92068F5
:100510008068C00707D0A06D3043A065E06D384308
:10052000E0650120F8BD20688068C007EAD100209E
:10053000F8BD0000E8FFFF7FF8B5044600200090FA
:10054000206802F0DFFC002845D120688168234A3A
:1005500010271140002930D18168D6433140491C11
:1005600081601F48006807218905084000020AD5FC
:100570001D481C490068FFF7BDFD401C00E0401EFF
:1005800000900028FBD1607E012824D001F09CF966
:1005900005461BE002F0B6FC002804D12068816803
:1005A0003140491C816001F08FF9401B02280DD9B0
:1005B00020680068C043C00708D0A06D3843A0651C
:1005C000E06D01210843E0650846F8BD2068016838
:1005D000C943C907DED10020F8BD00001700008024
:1005E00008270140400D03004400002010B52D4CA9
:1005F000012023881A464100615A994201D90B46CD
:1006000002E0914200D20A46401CC0B2FA28F2D35E
:10061000981A254C002802DD618C40186084E0792E
:10062000411CE17104283BD322200521205EFFF705
:1006300077FD1E4948431E49FFF772FD1A21615E8E
:1006400000B248430A21FFF76BFDA18B411801203E
:100650002056484360842082E078012803D0E07867
:10066000002803D004E0208A608201E0208AA08272
:1006700000206084E0711220205E0E49401849007D
:10068000884201D996200AE01220205E7D21FF30A9
:10069000C900F530884201D9642000E02820E082BA
:1006A00010BD0000C801002000000020E40C000084
:1006B000FF0F0000DC050000F8B504464088002567
:1006C0000A3080B2022160800A2802D96279002AA9
:1006D0000AD0962802D96279012A13D0E18888428B
:1006E00001D965716580F8BD0120607133202072E9
:1006F00065720091234621780833AC22204600F031
:1007000095F8F8BD61710720009023461C332178CD
:100710001E460022204600F04CF82079002802D026
:1007200025636563F8BD0621304600F0AEF8254626
:100730002035A9788842F5D1207F982108401828D3
:10074000F0D1607FA17F00020818E67F0002301818
:100750000009FFF7C6FD0E49FFF77AFD1327FF4397
:100760003946FFF7B2FD206330072978000D0818DD
:10077000697800020818FFF7B4FD0649FFF768FD25
:100780003946FFF7A2FD0449FFF75AFD6063F8BD43
:100790000000C842000048430000484202700022A6
:1007A0004271FF22F532914201D9C1807047C28067
:1007B0007047FFB581B0039800244F000A9D1E4684
:1007C000002813D002F031FBF8B202F0FEFA02F07A
:1007D0006DFB012800D10124039802F0F6FA02F023
:1007E00065FB012800D1641C02F03FFB02F01DFBF9
:1007F0007F1CF8B202F0E9FA02F058FB012808D198
:10080000641C06E06D1EE8B202F0AFFA3070EDB283
:10081000761C002D03D0002C01D1142DF2D302F050
:1008200024FB01980471204605B0F0BDFFB581B0EE
:100830001E460F4600250A9C02F0F7FA7806000EC5
:1008400002F0C3FA02F032FB012800D1012503981F
:1008500002F0BBFA02F02AFB012809D16D1C07E067
:10086000307802F0B2FA02F021FB641EE4B2761C8A
:10087000002D03D1002C01D0142CF1D302F0F5FA95
:10088000019928460D7105B0F0BD70B50446FF20F2
:100890000023312510E0227850400022060602D5C0
:1008A0004000684000E04000521CD2B2C0B2082AAA
:1008B000F4D35B1CDBB2641C8B42ECD370BD000034
:1008C00010B5024800F0C2FC10BD0000B4040020C6
:1008D00010B5034800F0BAFC024800F0B7FC10BDA8
:1008E000000600205C06002010B50446006C094993
:1008F0008008800040186064207814210838FFF7D1
:10090000F9FB04498031A164C106C90E0120884069
:10091000E06410BD000802400179084B8906890E89
:100920008A00D2180265054A4432491E42658A0788
:10093000920F01219140816570470000FC08024040
:10094000F0B5846CC56C6560046D002C02D0446DFC
:10095000856D65600B4F7C68056C1C263540012653
:10096000AE4034437C60046863608368102B036886
:1009700003D099600068C260F0BD9A600068C160F1
:10098000F0BD00000000024010B5012080F3108887
:10099000082000F05BFE002080F3108810BD10B529
:1009A000012080F31088802000F050FE002080F3AA
:1009B000108810BD72B6FEE703494A6901231B0483
:1009C000184302434A61704700200240044A5069BC
:1009D000044BC9001840014303480143516170476B
:1009E0000020024007E0FFFF0200010030B505498A
:1009F0004C6901252C434C610260BFF36F8F43604B
:100A000030BD00000020024030B50B4C002263696D
:100A10000125AD042B436361EFF3108372B620C947
:100A2000521C20C0D2B2402AF9D32069C003FCD4A2
:100A300083F3108830BD000000200240F8B507465F
:100A400000F042FFC51901242404114E03E000F018
:100A50003BFFA84214D230692042F8D130690D49D9
:100A600008400D49316103D00C4948600120F8BDB0
:100A700000F02AFFC41905E000F026FFA04201D3D0
:100A80000320F8BD30694003F6D40020F8BD000013
:100A900000200240FA830000FB830000B80600201B
:100AA000FEB50446002026460190403600900127FE
:100AB000307DFF070D46012810D0012030752068D9
:100AC00002F024FA00280BD0A06D20210843A06575
:100AD00001200190002030750198FEBD0220FEBD6E
:100AE000686802287ED02169B94202D06D4A9142DD
:100AF00007D120682968826A4903490B0A43826248
:100B00006DE0C3060F22DB0E1046216E9840814334
:100B10002868470302D0C7074BD102E04000C00E4F
:100B200048E0870701D5012044E0470701D50220AE
:100B300040E0070701D503203CE0C70601D50420AB
:100B400038E0870601D5052034E0470601D50620A8
:100B500030E0070601D507202CE0C70501D50820A5
:100B600028E0870501D5092024E0470501D50A20A2
:100B700020E0070501D50B201CE0C70401D50C209F
:100B800018E0870401D50D2014E0470401D50E209C
:100B900010E0070401D50F200CE0C70301D5102099
:100BA00008E0870301D5112004E0400301D512209D
:100BB00000E000209840014321666968E3698808E5
:100BC000401C98420BD820682F68836AC906C90E5A
:100BD0008A409343BA00120F8A401343836220680D
:100BE000AA6800E037E02968436909028B43114095
:100BF000490149090B4343612A68002A00DB69E780
:100C00002948016807239B051940284B9A4213D1B4
:100C10000B0211D4D202114302F084F92548244971
:100C20000068FFF767FA0C21401C484300E0401EB3
:100C300000900028FBD14DE71F4B9A4203D1CB0116
:100C400001D4920205E01D4B9A42D8D14A02D6D473
:100C50005A02114323E02069B84202D01149884268
:100C600006D120682968826A4903490B8A43826257
:100C70002A68002AC3DA0C48016807239B0519403B
:100C80000A4B9A4201D1D20208E00B4B9A4201D1A1
:100C9000920203E0094B9A42B1D15202914302F011
:100CA00041F917E70400008008270140001000B058
:100CB000400D030044000020004000B8002000B4B4
:100CC0007047704770470000FEB500260446029644
:100CD000374601960096002805D02546A06D2035A0
:100CE000002802D007E00120FEBD204600F0FCF8FD
:100CF000E7655420075520688168C900C90F12D1E3
:100D00008168724A114001221207114381607148C3
:100D10006F490068FFF7EEF94000801C00E0401EBC
:100D200000900028FBD120688168C900C90F08D154
:100D3000A16D10221143A165E16D01221143E1650E
:100D4000164602F0E3F8A16DC90601D4002804D0CC
:100D5000A06D10210843A065B4E0A06DFF21013112
:100D6000884302210843A065206802F0CBF80028E0
:100D70006DD1217EA06889030843617EA27EC903EC
:100D8000530319430843216B002901D001210903B2
:100D90000843E16808432169002902DA490049084B
:100DA00001E0012149050843297B490008430299D4
:100DB00008432978012909D1002A22D0A16D2022D7
:100DC0001143A165E16D01221143E165616A0029CA
:100DD00006D0FF23C1331940A26A014310460843DD
:100DE0002168CA683C4B1A400243CA606168019A94
:100DF000890F8907E06C0A4310432A7F012A04D037
:100E00000CE0012109040843E0E7636C226C491CF3
:100E10001A43A36C0B4311461943084321680A691E
:100E20002E4B1A4002430A610321606889078842F9
:100E30000DD0590788420AD04900884207D0284A75
:100E400091680F239B04994318400143916000214E
:100E5000626B206802F06DF82249A26B206802F0F4
:100E600068F80F212069C94300281CD001225205CF
:100E700090420AD12068826A227F9200121FD20615
:100E8000D20E9140226E1143816220684069616BED
:100E90004007400F88420BD1E765A06D80088000B5
:100EA000401CA0650FE02068826A0A438262ECE77A
:100EB000A06D0221884310210843A065E06D012147
:100EC0000843E06501263046FEBD0000E8FFFF7FD5
:100ED000400D0300440000200102FEFF02FCFF1F42
:100EE0000027014004FFFF0770B58CB005461421B0
:100EF0006846FFF742F9182105A8FFF73EF9244993
:100F00002868884242D1012080030590400409905E
:100F100005A800F0B9FD002801D0FFF74BFD1D48E2
:100F20000268012109050A430260006808400B902D
:100F300018484038416B012211434163406B002641
:100F400010400B900220009003200190052069467C
:100F50000296000700F004FC104C0F482060A660C9
:100F60000520E660606080202061400060618000B4
:100F7000A0612020E061C0012062204600F0C2F99B
:100F8000002801D0FFF716FD2C65A5620CB070BDDE
:100F9000002401404010024008000240B404002038
:100FA000F7B50446006801F0B1FF002845D1254699
:100FB0004035287D012840D001272F752068C16861
:100FC0001F4EC9070CD101F09DFF002804D02068F6
:100FD00081683140891C81602068C1683943C160E3
:100FE0002046FFF7A9FA002826D1A06D1549084030
:100FF000FF2101310843A0650020E065226D124900
:10100000D162226D11491163226D11495163226829
:101010001C2111602875206841681022114341602D
:101020002168206D4031029B019A00F0BDF92168D2
:101030008A683240121D8A60FEBD0220FEBD00009B
:10104000E8FFFF7FFEF1FFFF21040008B90400085C
:101050009F040008F8B5064604464036307D012856
:1010600007D0012737752046FFF7AAF9050002D0FF
:1010700028E00220F8BD206D2521095C022907D156
:1010800000F024F8050003D0A06D40210843A065BE
:1010900020684168102291434160002D204602D013
:1010A000FFF710FA09E0FFF70DFA050005D1A06D72
:1010B000FF21013188433843A0652068C168490891
:1010C0004900C160002030752846F8BDF0B5002801
:1010D00008D0014620314A79022A05D00422C26391
:1010E000002008710120F0BD026813680E24A3439C
:1010F0001360426C1468FF2301339C431460026840
:1011000014686408640014600C4E7268056C1C243A
:10111000254001242746AF403A437260826CC56C7B
:101120005560026D002A05D015689D431560826DDB
:10113000406D42604C7100200871F0BD000002401B
:10114000F8B50024014620314A79022A03D004214F
:10115000C16301242DE0026813680E25AB431360C0
:10116000026813685B085B001360426C1368FF251C
:101170000135AB431360104E7268056C1C231D4093
:1011800001231F46AF403A437260826CC56C5560C4
:10119000026D002A06D016681D02AE431660426D2D
:1011A000856D55604B7100220A71816B002900D05A
:1011B00088472046F8BD00000000024070B50400DA
:1011C00038D0206801684908490001601A4826683B
:1011D00014213018FEF78EFF800000252064356052
:1011E000164B5868216C1C22114001228A40104382
:1011F00058602046FFF778FB606C0560A06CE16CDE
:1012000041606068401E032807D82046FFF784FB32
:10121000206D0560606DA16D416025656565A56502
:10122000E56225636563A563E56320346571257117
:10123000002070BD012070BDF8FFFDBF000002401E
:10124000C06B70472030407970470000F0B42C4DDF
:101250002B6801680A68046C1C273C400426A640E1
:101260001E4211D056070FD50A68920603D40B68A8
:10127000042293430B606A68036C04213B4099404D
:101280000A436A60016B1CE00227A74006461F4024
:101290002036002F19D0970717D50A68920605D473
:1012A0000A680A239A430A60012171716B68026C13
:1012B0001C210A40022191400B436B6000213171D7
:1012C000C16A00291AD0F0BC08470827A7401F426E
:1012D00014D0120712D50A680E239A430A606A686E
:1012E000036C1C210B4001210C469C4022436A6088
:1012F000C163717100213171416BE2E7F0BC70474D
:101300000000024070B504003FD025482568142134
:101310002818FEF7EFFE80002064022026462036C3
:10132000707128681F4908402860A168E0686269F8
:101330000143206910430143A0690143E06901436F
:10134000206A014320680268114301602046FFF7CC
:10135000CBFA0121A06889030025884200D165608D
:101360002079616C8006800E0860A06CE16C4160A1
:101370006068401E03280AD82046FFF7CDFA206D8A
:101380000560606DA16D416004E0012070BD2565C0
:101390006565A565E563012070713571002070BD3C
:1013A000F8FFFDBF0F80FFFFF8B504468C462030E4
:1013B0000179002501290BD001260671477900210A
:1013C000012F07D08022E263017101252846F8BD74
:1013D0000220F8BD02274771E163206801684908CF
:1013E0004900016061462046FFF7AAFA206B0028F9
:1013F0002068016801D00E2205E0042291430160BB
:10140000206801680A2211430160606C0168084A83
:10141000C90302D5016811430160206D002802D084
:101420000168114301602068016831430160CDE724
:1014300000010000F8B51F4F044638780E46012819
:101440000AD001203870002078607D20C000FFF7AE
:10145000F5FA002802D029E00220F8BD04216160DD
:101460002268042A03D0491F3160A56814E00846A9
:10147000FFF7A2FA7D20C000FFF7E0FA16E0294648
:101480006068FFF7A3FA7D20C000FFF7D7FA0028B5
:1014900001D0356005E06D1CE268A1688918A94299
:1014A000EDD805494A6902239A434A6100213970FF
:1014B000F8BD0000B80600200020024005490120C8
:1014C0004A69C3071A434A614969002900DA0020C2
:1014D0007047000000200240F0B51FB4144E0546CE
:1014E0003078144601280AD00120307000277D2072
:1014F000C0007760FFF7A2FA002803D010E00220B6
:1015000005B0F0BD012D0DD021460198FFF77CFA02
:101510007D20C000FFF792FA06494A69AA434A6152
:101520003770EDE72246039B0198FFF75FFAEFE77C
:10153000B806002000200240064900204A69002A1F
:1015400007DA054A8A60054A8A604969002900DA93
:10155000012070470020024023016745AB89EFCD91
:10156000F0B5002255E0012393409E460B404FD03A
:1015700095082A4CAD002C19256E9607F70E0F26FC
:10158000BE403540AC4605252D07A84201D10025B7
:101590000FE0234DA84201D101250AE0214DA842C8
:1015A00001D1022505E0204DA84201D1032500E02C
:1015B0000525BD40654511D1184D80352F689F43E5
:1015C0002F606F689F436F60144D6F689F436F601B
:1015D0002F689F432F60236EB34323660468550032
:1015E0000323AB401C430460D408A4002418266ADB
:1015F0005507EF0E0F25BD40AE43266284689C431D
:10160000846044687546AC434460C4689C43C460CD
:10161000521C0B46D340A6D1F0BD0000001802407A
:101620000004005000080050000C005010B50828BD
:1016300008D105200821000700F032F9002801D167
:101640000149C87010BD00000000002070B5084DB1
:101650000446E868204203D0EC60204600F00AF817
:101660002869204203D02C612046FFF7DFFF70BDC0
:1016700000180240F8B505240746240740212046FB
:1016800000F00EF9344DA8728021204600F008F9D0
:10169000E87200240126802F22D0082F1FD12F4965
:1016A000032002F091FD05200821000700F0F8F862
:1016B000012814D1EE701220285E1421695EEA8A96
:1016C000401A032190423BDD287B401CC0B22873A6
:1016D000032801D3AC706C73FA2800D92973F8BDC4
:1016E000E87A0128FBD100F0EFF80746A86A381A1B
:1016F00008280DD27D21C900042002F065FD28795B
:10170000012805D1FF21F531022002F05DFD2C7189
:10171000AF62A87A012802D1687A401C6872287AE0
:10172000401CC0B228720528D9D9687A042801D390
:101730006E7002E00020C04368702C726C72F8BDBD
:10174000687B401CC0B26873032801D3AE702C7351
:10175000FA28F4D96973F8BD00000020881300004E
:10176000F0B500228EE0012595402B407ED00C790B
:10177000A407A40F012C01D0022C10D186685400BC
:101780000327A740BE43CF68A7403743876044681C
:10179000AC430D79ED06ED0F9540254345600C797E
:1017A000E443A40708D0C56854000326A640B54307
:1017B0008E68A6402E43C6600C79A407A40F022CA5
:1017C0000CD1D408A40027183D6A5407E40E0F2654
:1017D000A640B5430E69A6402E433E6205685400FC
:1017E0000326A640B5430E79B607B60FA6402E4392
:1017F00006604C68A403A40F43D09508244CAD00A8
:101800002F193D6E9407E40E0F26A640B54305261A
:101810003607B04201D100260FE01E4EB04201D182
:1018200001260AE01C4EB04201D1022605E01B4E03
:10183000B04201D1032600E00526A6402E43144DF8
:101840003E662C684E689C43F60200D51C432C6013
:101850006C684E689C43B60200D51C436C600C4D0E
:1018600080356C684E689C43B60300E009E000D503
:101870001C436C602C684E689C43F60300D51C43E7
:101880002C60521C0B681C46D44000D06BE7F0BDA6
:10189000001802400004005000080050000C0050E6
:1018A0000069084000D001207047426913460B4090
:1018B0001B0491430B4383617047002A01D081616F
:1018C00070478162704700000148806870470000DF
:1018D0003800002070B504000FD02168154808605A
:1018E00021681548086003CC41602068083C2168E5
:1018F0008860FFF7E9FF05460CE0012070BDFFF7A7
:10190000E3FF401B312805D92068C068400701D09B
:10191000032070BD2068C0684007F0D120680269CC
:10192000E1688A4201D0016101E0044901600020C0
:1019300070BD0000CCCC000055550000AAAA0000E4
:10194000006802490160002070470000AAAA000058
:101950000248816802788918816070473800002049
:1019600010B5084800240168821511430160032066
:1019700000F00AF8002801D0012401E000F028F866
:10198000204610BD0020024070B50F4E0024317873
:101990000546002915D07D20C000FEF7ABFB0146AF
:1019A0000A480068FEF7A6FB00F00CFC002808D1EE
:1019B000042D06D200222946401E00F03BF8756037
:1019C00000E00124204670BD3800002044000020C3
:1019D00008B5094801680122114301600068104000
:1019E000009005484038C26B01040A43C263C06BD3
:1019F0000840009008BD000040100240002809DBAC
:101A0000C106C90E0120884003490860BFF34F8F0B
:101A1000BFF36F8F7047000080E100E0002805DB16
:101A2000C106C90E012088400149086070470000C6
:101A300000E100E010B502F04BFB10BD10B50F4CFB
:101A4000216803225202914301432160C11FFF39E3
:101A5000FA390ED10A480621006848430949FEF7C1
:101A600049FB401C02E0002805D0401E6169490581
:101A7000F9D4002010BD032010BD0000007000400C
:101A80004400002040420F00FEB5044600250068D7
:101A9000524E2F46800359D5002001904F484038C0
:101AA000C06BC0000AD44D484038C26B01040A43E1
:101AB000C263C06B08400090012001904848016853
:101AC000821511430160FFF7FFFE009007E0FFF76A
:101AD000FBFE0099401A022801D903252CE040485A
:101AE0000068C005F3D5002D26D1F0690321090255
:101AF00008400FD0616981420CD0F06903210902CE
:101B0000F2698843012109040A43F261F2698A43B8
:101B1000F261F061C00759D0FFF7D6FE009006E0F1
:101B2000FFF7D2FE0099411A2E488142D5D8F069BC
:101B30008007F5D5002D49D02F460198002805D003
:101B400026484038C26B01048A43C2632078C0072C
:101B500005D0706961688008800008437061207852
:101B6000800606D57069032109038843A1680843EC
:101B700070612088400411D5706921698000800857
:101B800008437061012120698907884206D1134802
:101B90004038C168012212041143C1602088000549
:101BA00012D57069032189038843E1680843706195
:101BB0000121E0688903884206D108484038C1689D
:101BC000012212041143C1603846FEBDF0690321B1
:101BD0000902884361690843F061AEE740100240A2
:101BE0000070004088130000F8B50D46040044D092
:101BF0004D4800684007400FA84214D24A4F386849
:101C0000C008C00028433860FFF75EFE064605E0C6
:101C1000FFF75AFE811B4548814260D8386840076B
:101C2000400FA842F4D12068414E81070DD54007EE
:101C300004D5B068072109030843B060B0680F21DC
:101C400009028843A1680843B0602078C00731D0FA
:101C5000606801280AD002280BD000280FD0344930
:101C6000403103280ED0C969890704E0316889032F
:101C700001E031688901002906DB0120F8BD3168E7
:101C80004905F8E7096AEFE7B168C908C9000143E7
:101C9000B160FFF719FE074605E0FFF715FEC11B0F
:101CA000224881421BD8B068382108406168C900C9
:101CB0008842F2D11C4801684907490FA94216D948
:101CC0000168C908C90029430160FFF7FDFD074607
:101CD00007E0FFF7F9FDC11B1448814201D9032039
:101CE000F8BD114800684007400FA842F1D12078A4
:101CF000400706D5B168072000038143E06801432F
:101D0000B16000F031F8B1683C2289091140094AFC
:101D1000515CC906C90EC8400749086007480068F9
:101D2000FFF732FEF8BD00000020024088130000DB
:101D3000001002401C470008440000203C00002026
:101D40000648074900688968064A4904490F89001E
:101D5000515CC906C90EC84070470000440000200D
:101D6000001002405C47000810B5204CA068204AD3
:101D70008006400F16D0A0688006410F5010012940
:101D80000FD0A1688906490F022912D0A0688006E9
:101D9000400F042823D0A0688006400F032821D0DC
:101DA000002010BD206801218004400F81401046B2
:101DB00012E0E1688B07E1689B0F4906490F491C57
:101DC000032B00D01046FEF795F9E1684904490E4F
:101DD0004843E168490F491CFEF78CF910BD01200A
:101DE000C00310BD7D20000210BD000000100240A5
:101DF0000024F400F8B504007ED020783827C0070E
:101E0000E74E002845D0B068F16838408907890F4F
:101E1000102802D008280AD001E0032907D00121A8
:101E200060680904884209D13068084314E03068CA
:101E300080032ED560680028DED02AE00523012229
:101E40001B0492049842306802D110433060EBE7E3
:101E500088433060306890433060606800280CD060
:101E6000FFF732FD054604E0FFF72EFD401B642816
:101E700073D830688003F7D50BE0FFF725FD0546E2
:101E800004E0FFF721FD401B6428F1D8306880038F
:101E9000F7D42078800769D5B068F16838408A07A0
:101EA0000721920FC902102802D0002813D001E0A8
:101EB000022A10D0E068002846D0306888432169A3
:101EC000084330603168FF20013001433160FFF783
:101ED000FBFC05462CE03268520502D5E268002A78
:101EE0008AD072687F231B029A4363691B021A43DC
:101EF0007260002810D100E08DE0306888432169CD
:101F000008433060306801218004400F8140A548BB
:101F1000FEF7F0F8A4490860A4480068FFF734FD14
:101F2000002878D122E0FFF7CFFC401B02289FD881
:101F300030684005F7D570687F21090288436169E0
:101F400009020843706011E03168FF2001308143CD
:101F50003160FFF7B9FC054605E096E0FFF7B4FCF9
:101F6000401B022884D830684005F7D42078904D73
:101F700000072ED5B0688006400F03280AD0A0695C
:101F80000028286A16D0012108432862FFF79CFC2C
:101F900007460BE0286A80071BD5A06900289FD060
:101FA00017E0FFF791FCC01B02286ED8286A800753
:101FB000F7D50EE0400840002862FFF785FC074691
:101FC00004E0FFF781FCC01B02285ED8286A800766
:101FD000F7D4207840076AD500200090B0688006CA
:101FE000400F042818D0F06BC00008D4F16B01201A
:101FF00000070143F163F16B0140012000906D483F
:102000000168C90518D4026881150A430260FFF708
:102010005BFC07460CE083E0E869800747D5A068D1
:1020200000287DD043E0FFF74FFCC01B02282CD8CE
:1020300060480068C005F6D5A068012810D00421CA
:102040000528E86910D040084000E861E869884345
:10205000E861A068002814D0FFF736FC07460CE0C2
:10206000E86901210843F3E70843E861F8E7FFF76F
:102070002BFCC11B5048814265D8E8698007F6D522
:102080000DE0FFF721FC074606E05CE0FFF71CFCD3
:10209000C11B4948814256D8E8698007F6D40098A8
:1020A000002804D0F16B012000078143F163E0694F
:1020B000002873D0B1688906490F02294DD0012745
:1020C0003F060228306805D0B8433060FFF7FCFBBC
:1020D00004463AE0B8433060FFF7F6FB054604E0FB
:1020E000FFF7F2FB401B02282DD830688001F7D49F
:1020F000616A206AA26A0843E16A12021143084336
:10210000216B0843F1682D4A11400843F0603068A4
:1021100038433060F068012109070843F06000E0AF
:102120003AE0FFF7D1FB044604E0FFF7CDFB001BCC
:10213000022808D830688001F7D52FE0FFF7C4FBEC
:10214000001B022801D90320F8BD30688001F5D4B6
:10215000F0681B490840F06020E00128F4D0F068E6
:10216000226A8107890F914216D17021626A01406B
:10217000914211D17F21A26A0902014012029142CB
:102180000AD11F214904E26A0140914204D1400F63
:10219000216B4007884201D00120F8BD0020F8BD26
:1021A000001002400024F400440000203C00002005
:1021B0004010024000700040881300008C80C11F56
:1021C000FCFFFEEF094910B5401E884201D90120ED
:1021D00010BD074C60610321081F01F079FF00204A
:1021E000A06107202061002010BD0000FFFFFF005C
:1021F00000E000E070B5040005D025462035687F7A
:10220000002802D006E0012070BD0020287720467B
:1022100000F016F802206877211D206801F0DAF935
:10222000012240342272AA77EA7722706270A2708B
:10223000E27022716271A271E2716A77002070BD52
:1022400008B500680549884207D105480268C913E6
:102250000A43026000680840009008BD002000406A
:1022600040100240014620314A7F012A01D001205E
:10227000704702224A770168CB6801221343CB6082
:1022800000680949884202D00849884207D181681C
:10229000074B1940062905D0DB1F994202D001687F
:1022A0001143016000207047002C014000040040F1
:1022B0000700010010B586B0044614216846FDF7FA
:1022C0005CFF0E492068884215D10D48416B012200
:1022D00011434163406B6946104005901020009007
:1022E0000220019000200290039004200490052019
:1022F0000007FFF735FA06B010BD000000200040CF
:1023000000100240F8B50446002026462036009012
:10231000307F0D4601280CD00120082730770C2A89
:1023200048D008DC002A10D0042A1ED0082A06D182
:1023300030E00220F8BD102A52D0142A60D00120CB
:102340000090002030770098F8BD206801F08EF9E9
:102350002068816939438161206881690422914341
:102360008161206881692A6911E0206801F0BCF967
:10237000206881690122D20211438161206881694C
:10238000521091438161206881692A6912021143C8
:102390008161D6E7206801F0E7F92068C169394317
:1023A000C1612068C16904229143C1612068C1698B
:1023B0002A6912E0206801F017FA2068C169012239
:1023C000D2021143C1612068C269012189028A4396
:1023D000C2612068C1692A6912021143C161B0E774
:1023E000206801F037FA2068416D39434165206863
:1023F000426D04218A4342652068416D2A6912E0DA
:10240000206801F055FA2068416D0122D202114383
:1024100041652068426D012189028A434265206836
:10242000416D2A691202114341658AE770B50400C3
:1024300005D025462035687F002802D006E001201F
:1024400070BD00202877204600F016F8022068773B
:10245000211D206801F0BEF8012240342272AA77C3
:10246000EA7722706270A270E27022716271A271CA
:10247000E2716A77002070BD7047000030B50346F6
:10248000044600252033403000290CD004290CD00C
:1024900008290CD00C290CD010290CD0C278012AA4
:1024A0000BD0012030BD9A7FF9E7DA7FF7E7027899
:1024B000F5E74278F3E78278F1E70222002912D0AB
:1024C000042912D0082912D00C2912D0102912D0B8
:1024D000C270002911D0042914D0082916D00C2963
:1024E00040D001253CE09A77F3E7DA77F1E7027014
:1024F000EFE74270EDE78270EBE72068C3681343B3
:10250000C36008E02068C268042302E02068C26853
:1025100008231A43C2600122206801F099F8134988
:102520002068884205D0124A904202D0114A904257
:1025300004D1426C0123DB031A4342642068012268
:10254000884202D00C49884207D181680B4B194060
:10255000062905D0DB1F994202D0016811430160B2
:10256000284630BD2068C2681023D2E7002C014005
:102570000044014000480140000400400700010001
:1025800010B5014680310A79012A15D001220A715D
:1025900024228A6002681368146864086400146066
:1025A0000122520793430022426600680360202004
:1025B00088600A71104610BD022010BD7047704738
:1025C00070B5044605468034207901281AD00120D0
:1025D00020712420A0602868066802685208520012
:1025E00002602868826807235B069A430A43826078
:1025F000284601F08FF9286806602020A06000209E
:10260000207170BD022070BD70B50446054680344F
:102610002079012819D0012020712420A060286889
:102620000668026852085200026028688268D20078
:10263000D2080A438260284601F06CF928680660D7
:102640002020A0600020207170BD022070BD704766
:102650007047F8B504468034A1680546E66800680E
:10266000826810271206002A1BDA212919D1EFF3FC
:102670001081012282F31088826880239A4382604D
:1026800081F31088E86F002808D0FEF71FFD0028AE
:1026900004D0E86FFEF7D4FD202824D0284601F0AE
:1026A000DFFA2868816849061BD5222E19D1EFF37D
:1026B0001081012282F31088826840239A4382604D
:1026C00081F310882068002808D0FEF7FFFC00285E
:1026D00004D02068FEF7B4FD202804D0284601F07D
:1026E0008DFA0020F8BD27610320F8BD70B5040005
:1026F0001AD0242025468035A86020680168490842
:102700004900016020680026066020684660206855
:102710008660204600F0BAF92E61AE60EE60E66693
:1027200026672E71002070BD012070BD704700002B
:10273000F8B503680446D86919689A68B44D064626
:102740002E4025468035002E75D0B24EB24F164031
:102750000F4037436ED0C70706D0CF0504D50127F9
:102760001F622B693B432B61830708D5D30706D033
:10277000276802233B622B6904273B432B614307F5
:1027800008D5D30706D0276804233B622B690227AC
:102790003B432B61030709D520230B40334305D06E
:1027A0002668082333622E691E432E61030509D56E
:1027B0004B0107D501232668DB0233622B692026F3
:1027C00033432B612B69002B42D080060AD5202091
:1027D0000140C0050240114304D0616F002901D0BF
:1027E00020468847286921688968490602D428213B
:1027F000084232D0204601F001FA2068816849067B
:1028000027D5EFF31081012282F3108883684022DC
:102810009343836081F310882868002819D07F498A
:1028200081632868FEF78CFC002811D02868816B32
:102830000DE000E017E0860615D5012720263F07AA
:102840000E4017403E430ED0616FB5E020468847EA
:10285000F8BD2046FFF76AFFF8BD2046FFF766FF88
:1028600000202861F8BDE66E012E7DD1C6067BD51D
:10287000CE0679D510221A6220688168264649065C
:102880004036002949DA2B68196849680904090C9F
:10289000E8D0B78B8F42E5D9F183196809688906BA
:1028A00034D4EFF31081012383F3108803681701F8
:1028B000BB43036081F31088EFF31081012080F3A4
:1028C0001088206883685B085B00836081F3108850
:1028D000EFF31081012080F310882068836840277F
:1028E000BB43836081F310882020E8600020E0660D
:1028F000EFF31081012080F3108820680368934370
:10290000036081F310882868FEF7E0FB022020674F
:10291000B08BF18B401A81B235E0B18BF38BC91AC1
:10292000F38B89B2002B9DD000299BD0EFF310834D
:10293000012686F310880668FF272137BE4306600C
:1029400083F31088EFF31083012080F31088206850
:102950008668304FFF433E40866083F31088202016
:10296000E8600020E06600E011E0EFF310836067AC
:10297000012080F31088206805689543056083F383
:102980001088022020672046FFF718FEF8BDC60217
:1029900008D5560206D50120000518622046FFF72B
:1029A00057FEF8BD06060BD501278026FF050E4011
:1029B0003A40164304D0A16F002900D046E7F8BD85
:1029C000420614D54A0612D52046EFF310810122A3
:1029D00082F310881A684024A2431A6081F3108899
:1029E0002021A9600021816700F070F9F8BD020282
:1029F00005D54A0003D52046FFF729FEF8BDC001E2
:102A0000FCD50029FADA2046FFF7D9FDF8BD000011
:102A10000F0800000100001020010004893A00089E
:102A200070B5040005D025468035A868002802D07E
:102A300006E0012070BD00202871204600F048F813
:102A40002420A860206801684908490001602046E8
:102A500001F024F90128EDD0A06A002802D0204618
:102A600000F07AFF206841680922D2029143416058
:102A7000206881682A2291438160206801680122D0
:102A800011430160204600F0CDFF70BD10B5044633
:102A900000680C49884213D10B4801680122920357
:102AA00091430160C0210948FEF75AFD802000597A
:102AB000FEF784FBE06FFEF781FB1B20FEF79EFF15
:102AC00010BD0000003801404010024000040050DA
:102AD000F0B58DB0044614216846FDF74EFB182171
:102AE00005A8FDF74AFB3249206888425ED10120E3
:102AF00000260590069605A8FEF7C6FF002801D01F
:102B0000FDF758FF2B480268012189030A43026040
:102B1000006808400B9027484038426B02210A4366
:102B20004263406B6A4608400B90C02043C2039644
:102B3000694621480496FEF713FE214D1F48286080
:102B4000AE603220EE60686080206E61AE61470149
:102B50002F62EE6128612846FEF7D4FB002801D0E1
:102B6000FDF728FF80200551AC621448144D143045
:102B70005C352860332068601020EE60A8606E61CC
:102B8000AE612F628020EE6128612846FEF7BAFB15
:102B9000002801D0FDF70EFFE567002202211B206F
:102BA000AC62FEF747FF1B20FEF738FF0DB0F0BD0B
:102BB0000038014040100240000400501C00024058
:102BC0000006002070B58C231B58202B01D002205A
:102BD00070BD00290BD0002A09D00124836824038A
:102BE000A34206D10369002B03D1CB0701D00120FA
:102BF00070BD0023C36603685C6824020BD5EFF345
:102C00001084012585F310881D680126B60635431A
:102C10001D6084F3108801F0F7F870BD70477047AD
:102C200070B5054604468035A868202801D00220EA
:102C300070BD00290BD0002A09D00123A0681B0316
:102C4000984206D12069002803D1C80701D001208D
:102C500070BD2046403021658282C28200212961F8
:102C60002120A860E06F002819D0154BC362E36FE4
:102C700014481863E36F14485863E06F1346816388
:102C80002068E66F024628323046216DFEF78CFB45
:102C9000002804D0102028612020A860D7E72168F0
:102CA00040200862EFF31081012080F31088206833
:102CB000826880231A43826081F31088002070BDEF
:102CC000A53B0008F13B00089D3A0008704770479B
:102CD000FEE770B501240525E4022D0700222146F8
:102CE0002846FEF7EAFD6600002231462846FEF738
:102CF000E4FD022001F0C4FA012221462846FEF735
:102D0000DCFD022001F0BCFA002221462846FEF735
:102D1000D4FD012231462846FEF7CFFD70BD70B5C7
:102D200001240525E4022D07002221462846FEF74E
:102D3000C4FD0122160331462846FEF7BEFD0420DD
:102D400001F09EFA012221462846FEF7B6FD042036
:102D500001F096FA002221462846FEF7AEFD012238
:102D600031462846FEF7A9FD70BDF1B500240126C5
:102D7000F602052725463F07002231463846FEF772
:102D80009CFD022001F07CFA012231463846FEF714
:102D900094FD6006040E012109033846FEF780FD0C
:102DA000002801D0641CE4B2012001F069FA6D1C16
:102DB000EDB2082DE0D30098002803D0FFF789FF7B
:102DC0002046F8BDFFF7ABFFFAE7F8B50126052767
:102DD0000546F6023F07002231463846FEF76DFDF4
:102DE0000024E80901D0012200E0002201210903AA
:102DF0003846FEF762FD6806050E022001F040FA33
:102E0000012231463846FEF758FD022001F038FA1B
:102E1000002231463846FEF750FD022001F030FA1C
:102E2000641CE4B2082CDCD3F8BD70B50122052582
:102E300014032D0721462846FEF73FFD0122D60246
:102E400031462846FEF739FD042001F019FA002228
:102E500021462846FEF731FD042001F011FA002238
:102E600031462846FEF729FD70BD70B501240525C1
:102E7000E4022D07002221462846FEF71EFD6600CB
:102E8000002231462846FEF718FD042001F0F8F92B
:102E9000012221462846FEF710FD01223146284630
:102EA000FEF70BFD042001F0EBF970BDF8B501222F
:102EB000052516032D07002431462846FEF7FDFCA4
:102EC000012001F0DDF90122D70239462846FEF73C
:102ED000F4FC012001F0D4F907E0641CE4B2642C96
:102EE00003D9FFF7C2FF0120F8BD31462846FEF79F
:102EF000D7FC0028F1D1002239462846FEF7DDFC38
:102F00000020F8BD8068C007C00F70478068400788
:102F1000C00F7047C0680005800F01D000207047C7
:102F200001207047026807239B059A430A43026009
:102F3000704710B543690424214007248C40A34303
:102F40008A401343436110BDF0B53F4885B04188C6
:102F500080884EBA45BA06213B4801F05FF9010A64
:102F6000C0B2009039480191018A394B5980022141
:102F7000415699800179D980018B1981418B598102
:102F8000818B9981C18BD981018C1982817940799A
:102F9000090201432C4F7019803F59820A282DD80D
:102FA0002948009982798A4228D1C27901998A42B6
:102FB00024D101783970407878706800B8700324A3
:102FC00000200BE031184900595A0A123A55641C86
:102FD000E2B2B954521C401CD4B2C0B2A842F1D3E0
:102FE00019482146803801F019F93855641CE1B2BE
:102FF000000A7854491CC8B201F07AF9FF2E21D199
:10300000012D1FD11048009982798A421AD1C179C5
:103010000198814216D114220EA16846FDF794F85A
:1030200000246D4603E0285D3855641CE4B2684610
:10303000FDF7AEF8A042F6D86846FDF7A9F8C0B291
:1030400001F056F905B0F0BD480100200000002055
:10305000BC0300204443452D323330322D56352EEB
:10306000305F48414C000000F8B5664E0621B0883C
:1030700040BA04B2708845BA304601F0CFF8034632
:1030800000203246803A315C1154401CC0B2062800
:10309000F9D3D9B2180A91715B4FD0710F2D1CD0A2
:1030A000042D41D0594A5300052D58D0062D7ED00D
:1030B000072D7AD0082D0FD1B27991420CD1F17938
:1030C000884209D1032C07D820257D5F3C8401F07C
:1030D0007BFA00286AD03D84F8BDB3799942FBD1D0
:1030E000F1798842F8D1601EF6280CD8F889FC8165
:1030F000C5B201F069FA002801D0FD81F8BD7078F1
:1031000000280DD1F8BDFF20107150711446062122
:103110003C4801F083F8A071000AE0713078EFE7D5
:10312000082001F0E5F8F8BDB2799142FBD1F179C0
:103130008842F8D17D20C0008442F4D8388B3C838B
:1031400005B201F041FA002801D03D83F8BD082006
:1031500001F0CEF8388B2E4909684863F8BDB5797F
:10316000A942FBD1F1798842F8D1A0189842F5D84C
:103170001A257D5F20460A2148431021795EFCF71D
:10318000CFFF7883601F0F2800D87C831A20385E19
:103190000528E3DB1A20385E1428DFDC01F014FA7E
:1031A0000028BDD07D83F8BD01E012E021E0B579B3
:1031B000A942F8D1F1798842F5D1A0189842F2D805
:1031C0001C257D5FBC8301F0FFF90028A8D0BD83DA
:1031D000E9E7B2799142E6D1F1798842E3D1FD8BFA
:1031E000FC830C48786201F0F9F9002898D0FD833F
:1031F000D9E7082001F07CF82020385E00F002FFBB
:10320000D1E700004801002000000020E40C00008D
:1032100020050020D87700083EB50021184800910D
:103220000191164A029102600122D204816042603B
:10323000C1601203026104224261017641760124D9
:10324000847641620246C461203281621173072391
:10325000436301631177C164FDF736FD002801D097
:10326000FDF7A8FB07480090694601940448FDF764
:1032700017FC002801D0FDF79DFB3EBD0024014056
:10328000500400200200000408B50C48816B0122A4
:1032900011438163806B02211040009000220920BD
:1032A000FEF7C8FB0920FEF7B9FB002202210A2025
:1032B000FEF7C0FB0A20FEF7B1FB08BD001002407C
:1032C000F0B587B014216846FCF757FF3C48416BC6
:1032D000022631434163416B31400591416B012529
:1032E00029434163406B2A46284005900520354913
:1032F0000007FEF7E2FA0520002220210007FEF772
:10330000DCFA314F012211463846FEF7D6FA042086
:10331000002400900520029469460195039400075B
:10332000FEF71EFA082000903120000401900520CD
:10333000694602940007FEF713FA2020009005204A
:1033400069460396019502940007FEF709FA4020AA
:10335000009005200194694602940007FEF700FAE8
:1033600080200090112000040190052069460294FD
:103370000007FEF7F5F90095029469463846019575
:103380000394FEF7EDF90320C0020090112001AA7A
:1033900051C2052069460007FEF7E2F9002201212B
:1033A0000620FEF747FB0620FEF738FB002201212E
:1033B0000720FEF73FFB0720FEF730FB07B0F0BD0C
:1033C00000100240041800000004005010B5094825
:1033D00007490160032141600749C16007498160D5
:1033E000FEF778FA002801D0FDF7E4FA10BD0000DE
:1033F0000030004010050020FF0F0000B80B000057
:1034000010B588B01C216846FCF7B7FE174816496E
:1034100001600024022184604160046114498461D8
:10342000C160FEF7E7FE002801D0FDF7C3FA0F48A0
:10343000FEF7FCFF002801D0FDF7BCFA60200090E9
:103440007D20C00001900294002269460494074840
:10345000FEF758FF002801D0FDF7ACFA0348FEF74D
:1034600029FF08B010BD000000200040200500200A
:10347000E703000010B51848164901604B21C90147
:10348000416000218160C16001618161C1610162AF
:103490000C22416242618162FFF7C2FA002801D02A
:1034A000FDF788FA00210C48FFF7AEF8002801D09C
:1034B000FDF780FA00210848FFF782F8002801D0C4
:1034C000FDF778FA0448FFF75BF8002801D0FDF714
:1034D00071FA10BD003801406C050020FEE770470E
:1034E000704710B5FEF734FA00F002F810BD000086
:1034F00030B5184B58680124002804D05868401E85
:10350000586000D11C70144D00210C204843401914
:103510004268002A09D04268521E426005D14470B8
:103520000278012A01D182684260491CC9B2062989
:10353000EBD39868401C98609868084A0021904234
:1035400000D199605878401CC0B258700A2800D346
:10355000597030BD2C000020D0030020FFFFFF7FFA
:1035600030B591B034216846FCF707FE00240120F5
:103570000D940E940F9440021094FEF75FFA0A2007
:103580000090FF200130039040200590012006901C
:1035900008200A90022580030B90079500030494ED
:1035A0000C90089509946846FEF724FC002801D089
:1035B00072B6FEE707200D900F9402210E9510942D
:1035C0000DA8FEF711FB002801D072B6FEE711B07E
:1035D00030BD704770B50268184C194EA04201D03A
:1035E000B04204D1134670254A68AB431A43154BC9
:1035F000154DA04208D0B04206D0144EB04203D0C0
:10360000984201D0A84204D103263602B243CE68C4
:1036100032438026B2434E69324302608A68C262F6
:103620000A688262A04203D0984201D0A84201D128
:10363000096901630121416170BD0000002C014056
:1036400000040040004401400048014000200040C8
:1036500010B5C906C90E0123046A8B409C4304625D
:10366000036A8A401343036210BD0000F0B5026A8A
:10367000520852000262056A43688269164C174E6E
:10368000224092080C6892001443022295438A68F3
:10369000134F2A43B04204D0B84202D0114DA84281
:1036A00006D10825AA43CD681543042295432A462E
:1036B000B04204D0B84202D00A4DA84206D1032538
:1036C0002D02AB434D691D438B692B4343608461DD
:1036D000496841630262F0BD8FFFFEFF002C01408C
:1036E0000044014000480140F0B5026A10239A43AB
:1036F0000262046A43688269174D184E2A40032506
:103700002D02AA430D682D021543202294438A6896
:1037100012012243B04207D11446CA688027BC4335
:10372000120122434024A243B04205D00C4CA042D7
:1037300002D00C4CA04208D10324A402A3434C693C
:10374000A4001C438B699B00234343608561496847
:1037500081630262F0BD0000FF8FFFFE002C01407C
:103760000044014000480140F0B5026AFF230133E4
:103770009A430262046A4368C269174D174E2A4091
:1037800092080D68920015430122520294438A6800
:1037900012022243B04207D11446CA68C714BC4380
:1037A000120222430415A243B04205D00C4CA042A1
:1037B00002D00C4CA04208D103242403A3434C693B
:1037C00024011C438B691B0123434360C561496885
:1037D000C1630262F0BD00008FFFFEFF002C0140BC
:1037E000004401400048014070B5026A01231B03F8
:1037F0009A430262046A4268C369124D2B40032552
:103800002D02AB430D682D021D4301235B039C4336
:103810008B681E030C4B2643984205D00B4B9842F5
:1038200002D00B4B984206D101241346A4034A69E7
:10383000A34392011A434260C5614968016406626C
:1038400070BD0000FF8FFFFE002C014000440140CE
:103850000048014070B5026A01263604B243026294
:10386000036A4268446D0E4D2C400D682543740078
:10387000A3430C8924041C430A4B984205D00A4BED
:10388000984202D0094B984204D113464A69B34387
:1038900012021A434260456549688165046270BD41
:1038A0008FFFFEFF002C0140004401400048014012
:1038B00070B5026A01231B059A430262036A4268DB
:1038C000446D104D2C400D682D02254301246405E4
:1038D000A3430C8924051C430B4B984205D00B4B8A
:1038E000984202D00A4B984206D101261346B604EC
:1038F0004A69B34392021A43426045654968C1650B
:10390000046270BDFF8FFFFE002C014000440140A7
:1039100000480140F8B50446416E4034002915D0F6
:1039200000688168806809014D0F0A4E400F3746D4
:10393000315C083F385CC000FCF7DCFB6085785DDB
:10394000715DC000FCF7D6FB2085F8BD01206085C5
:10395000FAE700001447000810B5018DC90707D029
:1039600001684A6801235B049A43C36A1A434A60A8
:10397000018D890707D501684A6801231B049A4312
:10398000036B1A434A60018D490707D501684A68ED
:1039900001239B049A43436B1A434A60018D090734
:1039A00007D501684A680123DB039A43836B1A43F6
:1039B0004A60018DC90607D501688A6801231B0387
:1039C0009A43C36B1A438A60018D890607D5016843
:1039D0008A6801235B039A43036C1A438A60018D52
:1039E000490612D501684B6801221205446C9343C5
:1039F00023434B60416C914207D101684A6803231D
:103A00005B059A43836C1A434A60018D090607D50A
:103A100001684A680123DB04C06C9A4302434A6090
:103A200010BD0000FEB505460026803504462E6117
:103A3000FDF74AFF019020680068124F000709D582
:103A400001210097002249052046019B00F034FA2D
:103A500000280DD12068006840070BD50121009790
:103A6000002289052046019B00F026FA002801D09B
:103A70000320FEBD2020A860E860E66626672E7160
:103A80000020FEBDFFFFFF0110B5806A0022014645
:103A90004031CA83CA82FEF749FE10BDF8B5846A78
:103AA0002046803081680546C66820688068002707
:103AB0000006002806DA212904D1562007532046A3
:103AC00000F0CEF820688068400606D5222E04D18A
:103AD0005E200753204600F091F828691021084322
:103AE00028612046FEF722FEF8BD70B50146096840
:103AF000806A096800238906002937DB5E210B52A2
:103B0000EFF31082012181F3108801680C68FF2512
:103B10000135AC430C6082F31088EFF31082012171
:103B200081F3108801688C68640864008C6082F3FB
:103B30001088EFF31082012181F3108801688C68EE
:103B40004025AC438C6082F3108820228C210A50DF
:103B5000C16E01290AD1EFF3108281F31088016848
:103B60000C681025AC430C6082F310880367C16EAB
:103B7000012902D0FFF752F870BD5C21095AFEF707
:103B80001DFD70BD10B5806A01210167C16E01295C
:103B900002D0FFF744F810BD5C21095A4908FEF72E
:103BA0000DFD10BD10B501460968806A09688906D7
:103BB0001BD4002256210A52EFF31082012181F317
:103BC000108801688B688024A3438B6082F310887F
:103BD000EFF31081012282F310880068026840230D
:103BE0001A43026081F3108810BDFFF76FF810BD13
:103BF00010B5806AFFF76BF810BD000010B5EFF349
:103C00001082012181F3108801680B68FF242134A0
:103C1000A3430B6082F31088EFF31082012181F33C
:103C2000108801688B680D4C23408B6082F31088EC
:103C3000C16E01290AD1EFF3108281F31088016867
:103C40000B681024A3430B6082F3108820228C2180
:103C50000A500021C166416710BD0000FEFFFFEF62
:103C600010B5EFF31082012181F3108801680B6811
:103C7000C024A3430B6082F31088EFF3108201216C
:103C800081F3108801688B680124E405A3438B60ED
:103C900082F3108820218030816010BDF8B5044681
:103CA00081680069E26901436069002510430143AE
:103CB000206802684C4B1A400A4302602068416841
:103CC000032212039143E26811434160216AA06913
:103CD000014320688268454B1A400A43826020688D
:103CE000C16A626A090909011143C1624049206839
:103CF00088420FD13F4840698007800F10D00128CB
:103D000004D002280CD0032809D101E0042007E0E8
:103D1000082005E03849884201D1002000E0102049
:103D20000122E369D2033549354E364F93422AD1F9
:103D3000002806D0022807D0042807D0082843D13D
:103D400008E0FDF7FDFF03E00A4603E0FEF70CF88C
:103D500002003ED0606A4000315A1046FCF7CAF9B2
:103D6000616840004A088018FCF7C4F90146103920
:103D7000B94229D82349491C01400007420F206855
:103D80000A43C26025E0002806D0022807D0042894
:103D900007D0082818D108E0FDF7D2FF03E00A4653
:103DA00003E0FDF7E1FF020013D0606A4000315AE2
:103DB0001046FCF79FF961684A088018FCF79AF9E9
:103DC00001461039B94201D9012502E0216880B2CB
:103DD000C860204601214030418501850020606790
:103DE000A0672846F8BD0000F369FFCFFFF4FF117C
:103DF0000038014040100240004400400024F4001C
:103E0000F4460008EFFF000070B5044681654030BD
:103E1000002125468283803529612220E8602868B8
:103E2000002819D0214BC3622B68214818632B68E6
:103E300020485863286813468163A66D216832467E
:103E400024312868FDF7B0FA002805D01020286139
:103E50002020E860012070BD206900280CD0EFF31D
:103E60001081012080F3108820680268FF2301334D
:103E70001A43026081F31088EFF31081012080F370
:103E800010882068836801221343836081F31088BF
:103E9000EFF3108182F310882068826840231A4370
:103EA000826081F31088002070BD0000EB3A0008AA
:103EB000853B00089D3A0008FFB581B005460F46D6
:103EC000044680350A9E54E0701C52D0FDF7FCFC7D
:103ED0000499401AB0422FD8002E2DD020680168D6
:103EE000490746D5C069C043000542D40120216876
:103EF000C0020862EFF31081012080F3108820686F
:103F00000268FF23A1339A43026081F31088EFF324
:103F10001081012080F310882068826852085200C6
:103F2000826081F310882020A860E860286100206A
:103F30002871032005B0F0BDEFF31081012080F35C
:103F4000108820680268FF23A1339A43026081F33E
:103F50001088EFF31081012080F3108820688268B8
:103F600052085200826081F310882020A860E86027
:103F7000DDE72068C1693846884305D000200399F1
:103F80008842A1D00020D5E70120F8E710B51848F5
:103F9000FEF7CEFB1648FEF75CFB154C2068C069A7
:103FA000C043C0061DD42046FEF753FB21681020F5
:103FB0000862104C207800280ED10F480068406835
:103FC0008021081A207022780C490D48FCF7BCF8B3
:103FD00021780A48FCF7D1F8802208490448FEF706
:103FE000F1FD802205490248FEF7ECFD10BD0000FE
:103FF0006C05002000000020000600204800002082
:104000004801002010B504461F48FEF76FFB1E490B
:104010001E4808604B20C0014860012C02D0022CD1
:1040200003D005E04B20000201E0E12000024860DF
:1040300000208860C86008618861C86108620C223D
:1040400048624A6188621048FEF7EAFC002801D005
:10405000FCF7B0FC00210C48FEF7D6FA002801D08E
:10406000FCF7A8FC00210848FEF7AAFA002801D0B6
:10407000FCF7A0FC0448FEF783FA002801D0FCF707
:1040800099FC00F057F910BD6C0500200038014084
:1040900010B50D480D4A0178D3894078994202D174
:1040A0001378082B05D0002902D11178082902D0F5
:1040B00010BD032804D00628FAD1FEF7D5FF10BDA5
:1040C000FEF742FF10BD0000480100200000002064
:1040D0008307FF22DB0E9A408907090E99400028CA
:1040E00008DB830809489B001818036893430B43B7
:1040F000036070470007000F0838830804489B00DE
:104100001818C36993430B43C361704700E400E090
:1041100000ED00E002E008C8121F08C1002AFAD131
:1041200070477047002001E001C1121F002AFBD137
:1041300070470000062806D20C2148430549401864
:104140004178012901D000207047002141700120F1
:1041500070470000D003002070B50020154B0446C6
:104160000C2141430A46C9184C608C604C709C5429
:10417000401CC0B20628F3D30F487D21C900006857
:10418000FBF7B8FF0D49401E884201D901200CE021
:104190000B4948610B480722C3691B021B0A4D04E7
:1041A0002B43C3618C610A610020002800D0FEE728
:1041B00070BD0000D003002044000020FFFFFF007E
:1041C00000E000E004ED00E0062800D3FEE7012255
:1041D00082F310880C22064B5043C2185160916044
:1041E0000021517001221A5481F310887047000099
:1041F000D0030020062800D3FEE7012181F31088B8
:104200000C21054B00224843C1184A604A701A54D9
:1042100082F3108870470000D003002030B50346B9
:104220000B480C4C0DE01A78504000225B1CC5076F
:1042300002D04008604000E04008521CD2B2082A78
:10424000F5D30A46491E89B2002AECD130BD0000E0
:10425000FFFF000001A0000000280ED0012800D1BF
:104260000220012181F31088044948600020087071
:1042700080F3108808780128FCD170472C000020BA
:10428000F8B50D4E0746756900240D480B490068C6
:10429000FBF730FF7843B1690246B0698842FCD031
:1042A000884201D2091A01E02B1A59180C1901464B
:1042B0009442F2D3F8BD000000E000E040420F005D
:1042C00044000020FDF74CFBFFF74AF9FFF744FFDD
:1042D000FEF7F6FFFEF7D8FFFEF79EFFFFF790F818
:1042E000FFF7C8F8FFF772F800F03AF8FEE70000B1
:1042F00070B5052504462D07012220212846FDF72B
:10430000DCFA224608490948FEF78AFC0848FCF70F
:1043100099FF0128FAD10520FFF79EFF00222021F6
:104320002846FDF7CAFA70BDC80000206C050020C1
:104330005C06002010B508490868026810231A437B
:1043400002600968502008627D2138220901034873
:10435000FCF724FA10BD00006C05002018040020B2
:10436000FFF7E8FF804981480A8802800288804C74
:10437000002A02D00288A24201D1012202807D4897
:104380004A8802800288002A02D00288A24202D112
:104390007D22D20002800088774A126850637748F5
:1043A0008A8802800288002A03D00022825E521C82
:1043B00001D10A2202807248CA8802800288002540
:1043C000002A02D0425F521C00D1058008896D4945
:1043D00008800888002803D00020085E401C00D117
:1043E0000D800020085EFFF70DFE6748674B5E4FAB
:1043F000674C303F01461860088820800889228871
:10440000002A03D026885A4A964200D125800028E7
:1044100002D0574A904200D100202288904205D90C
:10442000B94203D8208008311960E5E75248FDF70A
:1044300019FF00215048FEF721F85648FEF709F908
:10444000802255495348FEF7BDFBFA225349544890
:10445000FCF7A6FD0520002220210007FDF72DFA1C
:1044600032210020FFF7B0FEFF21F5310120FFF7D8
:10447000ABFE4C490320FFF7A7FE7D21C9000420B5
:10448000FFF7A2FE0A210520FFF79EFE002600206E
:10449000FFF750FE002809D04148FCF7DBFDFCF790
:1044A000A5F8FA223D493E48FCF77AFD0120FFF7C6
:1044B00041FE002806D03C48FDF742FA01213B4866
:1044C000FDF7F3F90220FFF735FE002815D0761C22
:1044D0000520B6B204210007FDF7E7F9E12040010D
:1044E00086420AD92088401C2080218820488142A9
:1044F00000D1258000F072F800260320FFF71AFE95
:10450000002802D02A48022101700420FFF712FE81
:1045100000280BD00220FFF76DFE052001220421A8
:104520000007FDF7CAF92349012008700520FFF7AD
:1045300001FE002810D02048FCF7BEF81E4F787905
:10454000022809D1386BFBF7D3FE1C490870786B41
:10455000FBF7CEFE1A4908701A4F3878002896D01B
:10456000FFF796FD3D7092E7007800080E000020EE
:10457000FFFF000018000020200500201A00002086
:104580001C000020200000200070000824000020F3
:104590001E0000206C05002048000020C8010020FB
:1045A0005004002088130000100500200004005073
:1045B0000200002004000020180400200600002053
:1045C000050000200000002010B5012080F31088B5
:1045D00000F03CF8002181F3108810BD10B586B0C2
:1045E00002200090042001900E2002900120144C23
:1045F0000390606A08306062FCF79EFF1149606AB0
:1046000088420CD91048606204A96846FCF712FF82
:10461000002804D0FCF752FF012006B010BDE28B49
:1046200000230120616AFCF757FF002803D0FCF744
:1046300045FF0320F1E7FCF741FF0020EDE7000014
:1046400000000020D87700080070000800B589B08D
:10465000002000900190029003900220049004201A
:1046600005900F200690012007902048C1896A46D6
:104670001170C189090A5170018B9170018B090A6F
:10468000D170418B1171418B09125171818B9171E4
:10469000818B0912D171018C1172008C0012507241
:1046A000FCF74AFF08A904A8FCF7C4FE002804D0C0
:1046B000FCF704FF012009B000BD0D490120019B5A
:1046C000009AFCF709FF002808D1094901200831A8
:1046D000039B029AFCF700FF002803D0FCF7EEFED4
:1046E0000320E8E7FCF7EAFE0020E4E700000020F2
:1046F00000780008010002000400060008000A001B
:104700000C001000200040008000000101010103A6
:104710000701000008040204080101010000000074
:104720000000000000000000000000000000000089
:104730000000000000000000000000000100000078
:10474000020000000300000004000000060000005A
:104750000700000008000000090000000000000041
:104760000000000000000000000000000100000048
:104770000200000003000000040000009C47000845
:10478000000000204800000014410008E447000831
:1047900048000020900A00002441000800010100A8
:1047A0000100000000000000000000000000000008
:1047B00000004600000000000000000000000000B3
:1047C0000070000800000000000000000000000071
:1047D00000000000010000000400000000000000D4
:0447E0000024F400BD
:04000005080000C12E
:00000001FF
